:020000040000FA
:0600000070EF0FF012008A
:06002A000100221F00008E
:08003000CA00000002000000FC
:08003800EB0ED76EDB0ED66E55
:10004000F2941200F2A4FED71200C7D982E90F0E73
:1000500000140A0A13E0040A11E0070A0DE0020A7C
:100060000BE0060A09E0020A07E0090A07E0030AB2
:1000700005E0020A05E102D0010E03D0000E01D016
:10008000000E41E9E7CFD9FF1200A7D9C1D9AFECE3
:1000900008F0016E015021E0A5D9150EE66E4C0E58
:1000A000E66E030ED9D9030E00019E5D3BE1550EAD
:1000B0009F5D38E1A051026EA151036E93D9C60E27
:1000C000E66E60EC0FF041E90001010E9E6FA11D8C
:1000D0009F6FCCD9016E015003E10001028322D051
:1000E000150EE66E0D0EE66E010EB3D99E051AE1F1
:1000F000CC0E9F5D17E176D9080E035C03E0940EE9
:10010000035C04E10001028102970CD08F0E035CB6
:1001100009E102EBE6FF99DF41E9000903E0000194
:100120000281028744E9E7CFD9FF120056D970D97E
:10013000BBEC08F0016E015003E10001028339D0ED
:10014000020EE66EE66AFA0EE66E1E0E7DD96CD9D8
:100150003FD906EC0BF042E989D9320EE66E4C0E1F
:10016000E66E080E79D9050E00019E5D22E39F51CF
:1001700002E1030E0BD0C00E9F1502E1020E06D065
:100180003F0E9F1502E0040E01D0050E026E0250D4
:1001900039D9EF50C1080DE1022834D9EF50036E70
:1001A00003EBE6FF52DF41E9000903E000010281B1
:1001B000028744E9E7CFD9FF12000FD982E9020E86
:1001C000E66E1F0EE66ED5EC09F042E9005002E142
:1001D0005CDF06D0000403E058DF000102A1A6DFC7
:1001E000000102A111D028DF0001AA690001066BFD
:1001F000020E005C07E10E0EE66E1F0EE66EC8EC06
:1002000003F042E9000E05D002A302D0080E01D08F
:10021000070E41E9E7CFD9FF1200DFD881E941E8B5
:10022000000102A709D0020EE66EE66A000EE66E35
:100230001F0E0AD9F9D80BD0040EE66EE66AFC0E42
:10024000E66E1E0E01D9C4D8EAEC0AF042E9F5D8F0
:10025000016E015008E0150EE66E0D0EE66E0B0EF7
:10026000F8D89E5102E10001062BE6DE42E9E7CF15
:10027000D9FF1200F6D80C0EFED8FAEF01F0ADD877
:1002800081E941E8016A0C0EF36EF46AF350015CF7
:10029000000EF45405E20150B5D8EF6A012AF3D7F5
:1002A00042E9E7CFD9FF1200000102A117D00651A1
:1002B000050802E202911200FF0E0001AA5D04E1AE
:1002C000CE6ACF6A9E9008D09EA002D0AA2B9E90A4
:1002D0001D0EAA5D01E21200AA6B9FDF1200CE6A1A
:1002E000CF6A9E900001AA6B0001066B120075D8C0
:1002F00083E944E8056A00EBE6FF01EBE6FF11EC59
:100300000DF042E9000902E1010E5ED0000102B1E8
:100310000AD0020EE66E51DF41E9036E000102B120
:1003200002D0035051D054D800EBE6FF01EBE6FFBA
:100330003EEC0DF044E9000102B705D049D8EAECE3
:100340000AF042E901D070D878D8036E035002E178
:100350000C0E3AD0046A640E045C2FE2150EE66EB1
:1003600001C0E6FF0B0E75D89E5127E0050E9E5D7D
:1003700002E2040E29D0000100B514D029D831ECD6
:100380000BF042E900019E5102E1050E1DD0000173
:1003900002B704D01DD81AEC0BF003D019D885ECA5
:1003A0000BF042E95ED89EC0E6FF9F0EE66E000E9F
:1003B000E66E20D8042A052ACED7055002E1060EA3
:1003C00003D08DDF39DE090E45E9E7CFD9FF1200F2
:1003D0009E0EE66E000EE66E1200D9CFE6FFE1CF6C
:1003E000D9FF12000C0EE66E1F0EE66ED5EC09F07A
:1003F00042E9120082EC0DF045E933D8D8EC03F065
:1004000042E91200EA6A9E0FE96E000EEA2212002B
:1004100081E943E8000102910297029312005FEC28
:1004200008F045E900011200E66A030EE66E000ED0
:1004300022D846EC0BF045E91200CADF06EC0BF0BF
:1004400042E900DE36EF02F016D821EC0AF046E968
:10045000120011D80FEF02F00ED85FEC08F045E95A
:100460001200070EE66E000EE66E1200B1DF27ECFA
:0C04700008F042E91200E66EE8EF01F02F
:04047C0000010091EA
:100480000093009500970D0E016F306BC00E036F47
:10049000330E046FF10E056F3FEF01F00001029182
:1004A0003EEF02F09BD946E8C3D9076EF450086EC0
:1004B0000A0ED89008BE03D0075C000E085815E35A
:1004C000083404E207500D08000E08540EE389D9E1
:1004D000030E035C0AE1C00E04140001036F05EB78
:1004E00004F006EB05F0000E01D0010E47E9E7CF5E
:1004F000D9FF120073D9000E97D170D944E898D96A
:10050000056EF450066E060ED89006BE03D0055C4C
:10051000000E065813E3063404E205500708000EE7
:1005200006540CE35ED9030409E104EB01F0000179
:10053000015102E14C0E016F000E01D0010E45E9A0
:10054000E7CFD9FF12004AD96FD184D984E941E8B5
:10055000046A0250130A61E0010A5BE0030A55E0F5
:10056000010A50E01E0A4BE0020A47E0070A42E097
:10057000010A3DE01E0A39E01D0A50E0010A32E09E
:100580000F0A2DE0080A26E0090A21E00B0A1CE008
:10059000080A17E0010A12E0070A0DE0010A09E063
:1005A000030A03E0010A3EE03BD03AEC01F0090EF9
:1005B00038D064DF37D00001009334D000010083CD
:1005C00031D0000100912ED0000100812BD0010E0E
:1005D000E66E01D0E66ADDEC00F041E922D00001D0
:1005E000009520D0000100851DD00B0E1AD000010F
:1005F000009718D00001008715D0010E12D0E9D85D
:1006000051DF05D0E6D876DF02D0E3D876DF42E9C5
:1006100008D0DFD898DF42E905D040DF0A0E01D0CC
:10062000010E046E045042E9E7CFD9FF120012D93F
:1006300082E90050090A44E0050A38E0040A32E081
:100640000F0A2CE0010A26E0030A20E0010A1AE062
:100650000F0A14E0010A0EE0080A10E0020A06E0A0
:10066000010A28E1940EE66E1B0E27D0960EE66E68
:100670001B0E23D0990EE66E1B0E1FD0640EE66E85
:100680001B0E1BD0B00EE66E1B0E17D0BB0EE66E17
:100690001B0E13D0C70EE66E1B0E0FD0CF0EE66EEC
:1006A0001B0E0BD0D50EE66E1B0E07D0DE0EE66ECF
:1006B0001B0E03D0E70EE66E1B0EE66E69D842E90C
:1006C000750EE66E1D0EE66ED5EC09F042E9ACD073
:1006D00085D84AE808687DD8D5EC0AF042E900EBF5
:1006E000E9FF01EBEAFFEF5005E1300E006E000E6E
:1006F000016E08D06ED8300EE66E000EE66E6EEC1F
:100700000AF044E9020EE66EE66A720EE66E1D0E0F
:10071000E66E94D805E05DD877EC01F042E929D087
:100720000A6A150EF36EF46AF3500A5C000EF45474
:100730001BE26AD8B3EC0AF042E9BDC0C5F0BEC006
:10074000C6F0BFC0C7F00001C5510B6EC6510C6E9C
:100750000BEBE6FF0CEBE6FF57D870D803E18AEB12
:1007600008F002D00A2ADDD734D808EBE6FFEDDE28
:1007700043E9096E09EBE6FF5ADF41E94BE9E7CFB0
:10078000D9FF120000010291029778DE05EF08F010
:1007900025D81FD8070EE66E000EE66E8FEC0AF025
:1007A00044E9070EE66E000EE66E02D842E93CD040
:1007B00015D8700EE66E1D0E47D8000100A704D0B4
:1007C0006E0EE66E1D0E40D804D8C2EC09F042E968
:1007D0002BD000EBE6FF01EBE6FF12003BD883E9EC
:1007E0001200D950030FE66EDACFE6FF040E0001C7
:1007F0000024C56F000E0120C66FC5C0E6FFE66E7F
:100800003EEC0DF044E91200F76A0A34FE0BF66E76
:10081000F736F50EF6261B0EF7220900F5CFE6FF98
:100820000900F5CFE6FF120041E9E7CFD9FF12003A
:10083000D0DFA5EC0AF042E9F3501200CADF04EC65
:100840000AF046E900091200E66EC3DF41EC0AF047
:0E08500044E91200D9CFE6FFE1CFD9FF120034
:02085E00040193
:1008600020511F0B010801E012002051600BE842EB
:10087000E842E842E842E842010801E0120024515F
:1008800003E0240501E012002151230A39E0010AA6
:1008900033E0030A25E0010A1CE0240A31E0070ADC
:1008A0002FE0010A2DE0030A0EE0010A01E0120028
:1008B00031D90001960EB76F000EB86F0001C293D8
:1008C0000001080E17D026D90001960EB96F000E50
:1008D00005D020D900018B0EB96F000EBA6F12003F
:1008E00019D900018B0EB76F000EB86F0001C293CB
:1008F0000001070EBB6F12000DD922C492F0120046
:10090000120000018B6BC20E8C6F010E8D6F8E6B0F
:100910008F6B906B080E916F846B836B1A0E726EE7
:100920001E0E736E0401300E166F040E176F400E0C
:10093000146F0401196F380E1A6F040E1B6F880EA6
:10094000186F0401780E1E6F040E1F6F400E1C6F8F
:100950001200E4D884E90001836B040118BF24D09D
:100960000050195D02E21951006E0001836B0050C6
:10097000835D13E28351EA6A380FE96E040EEA22BE
:10098000EF50E66E83510124E96E000E0220EA6EFC
:10099000E552E750EF6E832BEAD70401400E196F42
:1009A0001817187D880E18130001835141E9E7CF0D
:1009B000D9FF12009ED812E1036AA1D802E1F450D7
:1009C00009E000EBE9FF01EBEAFF002A000E01223B
:1009D000EF50F3E176D88A6B010E846F97D089D8F7
:1009E00013E1036A8CD802E1F4500AE000EBF6FF51
:1009F00001EBF7FF002A000E01220800F550F2E19A
:100A000060D8010E8A6F846F81D088D881E941E86F
:100A100004011CBF55D0030E0001845D01E1846B0D
:100A200084514EE0020E845D03E104011D6B3FD052
:100A3000840540E189510001C56FC66BC55140086E
:100A4000000EC65502E2400E02D000018951016E2F
:100A500001EB1DF401500001895D896F780E876FED
:100A6000040E886F8A050AE1015011E085C0F6FF87
:100A700086C0F7FF0800F55030D8F6D7015007E0E0
:100A800085C0E9FF86C0EAFFEF5027D8F7D70001FD
:100A9000895110E104011D510001C56FC66B400E64
:100AA000C51905E1C65103E10001020E02D00001A3
:100AB000030E846F400E04011C171C7D880E1C134E
:100AC00025D00350005E000E015A00EB85F001EBCB
:100AD00086F003040001896F120087C0E9FF88C017
:100AE000EAFFEF6E872B000E8823852B86230106F5
:100AF000120014D883E941E8000184511200032A4E
:100B0000FF0EF36EF46AF3500318120042E9E7CFC8
:100B1000D9FF12000001030EB66F1200D9CFE6FF15
:060B2000E1CFD9FF120035
:0A0B260004012051600BE842E84290
:100B3000E842E842E842000901E012002151070AB8
:100B40003FE00B0A3DE0070A32E0010A23E00B0A0E
:100B50001FE0020A1DE0030A19E0080A10E0010A7A
:100B60000CE00F0A08E0030A01E0120015D90001A9
:100B7000040EC16F1200E1EF05F018EF06F00CD97A
:100B80000001C30EB76F000EB86F0BD039EF06F03F
:100B90006BEF06F005D90001B86BC40FB76F000EFC
:100BA000B8230001C2930001010EBB6F1200F8D8F8
:100BB000EA6AC40FE96E000EEA2222C4EFFF1200B7
:100BC0001200800E0401205D32E12351030A1FE070
:100BD000010A0AE0030A29E1DFD800011F0EB76FFE
:100BE0001C0EB86F120E1ED0C1D8C00EF6261C0EF9
:100BF000C6D8020E0001F76AB725F66EB851F72283
:100C00000900F5CFBBF00A00F5CFBCF00ED0AED88E
:100C1000C40EF6261C0EB3D8B7C0F6FFB8C0F7FF57
:100C20000800F5500001BB6FBC6B0001C2831200CD
:100C3000B3D80F0EE66E710EE66E0F0EE66EFFEC89
:100C40000CF043E9010EE66EC40EE66E000EE66E91
:100C5000FFEC0CF043E922C4C3F00401225104E18B
:100C60000001050EC16F12000001060EC16F81EF79
:100C700004F00401286B296B040120511F0B020AA8
:100C80000FE0030A0BE0010A18E186D8040128816D
:100C90000001C2A112D0040128830FD07DD80DD04D
:100CA0004BD801E0010E56D8B9C0E9FFEA6EEF500B
:100CB000040B03E00401010E286F0001B6050AE1F0
:100CC0000001280EB76F040EB86F0001C293000137
:100CD000020EBB6F1200040122050EE120511F0B12
:100CE00000090AE159D8030E0401215D03E1000166
:100CF000C28102D00001C291040122511CE12051A5
:100D00001F0B020818E124510F0B000914E014D83E
:100D100001E0010E1FD8030E0401215D04E1840EE1
:100D200036D8EF6E120024AF03D031D8EF6A12002C
:100D3000880E2DD8EF6E120033D80F0B080DF3502C
:100D40000001C66B000FC56F040EC62304012451B9
:100D5000800B1200040DF3500001C5250001B96F8E
:100D6000000E0001C6210001BA6F120015D804015F
:100D70002251F66EF76AD890F636F7361200F7224F
:100D80000900F5CFB7F00A00F5CFB8F01200B9C0EE
:100D9000E9FFBAC0EAFF12000001010EB66F1200AF
:080DA000FBDF040124511200E5
:080DA8006C500BE10401005145
:100DB0003C0BE842E8420D0802E1E6EF06F016EFD0
:100DC00007F0040E6C5C01E140D8120010D941E834
:100DD0000001B56BB66BBB6BBC6B93EC05F0016AA5
:100DE000010EF36EF46AF350015C000EF45419E244
:100DF0000001B65116E1F76A0134FE0BF66EF736C4
:100E0000CC0EF6261C0EF7220900F5CFC5F008001F
:100E1000F5CFC6F0C6C0FAFF0001C5511400012A83
:100E2000DFD794D842E9E7CFD9FF1200020E0001C4
:100E3000B55D09E161D8040100BD02D0C80E01D042
:100E4000880E006F1200DFEF07F0040E0001C15D95
:100E500009E122C46EFF6E50000802E2050E01D0C7
:100E6000030EC16F0001B50509E10AD8040104BDF4
:100E700002D0C80E01D0880E046F1200DFEF07F019
:100E8000B6D842E80001080EBB5D000EBC5905E271
:100E9000BB51016EBC51026E03D0080E016E026A96
:100EA0000401049304910250041301EB05F4015072
:100EB0000001BB5F0250BC5B280EB96F040EBA6F15
:100EC0000001C2A30BD00150021012E0B7C0F6FF20
:100ED000B8C0F7FF0800F5507AD8F5D701500210D6
:100EE00007E0B7C0E9FFB8C0EAFFEF5070D8F6D707
:100EF00043E9E7CFD9FF12007AD842E8030E040194
:100F00000015026E0151016EBB0EE96E000EEA6E15
:100F10000001EE500124BB6FED500220BC6F280E83
:100F2000B76F040EB86F015002100CE0B7C0E9FFB4
:100F3000B8C0EAFFEF50B9C0E9FFBAC0EAFFEF6EF0
:100F40005CD8F1D743E9E7CFD9FF12006D980001D3
:100F5000B65105E144D8840E006F04011DD0040190
:100F600020AF1CD00001BB510401265D0001BC5123
:100F70000401275904E226C4BBF027C4BCF080DF7B
:100F80000001010EB56F2BD8800E006F0401280EF2
:100F9000066F040E076FC80E046F12000001020EE8
:100FA000B56F0401056BC80E046F0401080E016FD4
:100FB000280E026F040E036FC80E006F12000001AE
:100FC000B56B0DD8880E006F0401046B1200B9C018
:100FD000E9FFBAC0EAFFEF6E0001FDEF07F0040180
:100FE000080E016F200E026F040E036F1200D9CF9E
:100FF000E6FFE1CFD9FF81E91200B92B000EBA2339
:0A100000B72BB8230106025A1200B4
:06100A00080EB86E400E56
:10101000E66E020EE66E3C0EE66EEFEC0EF043E975
:101020001200F2D882E9FE0ED76E880ED66EF294C8
:101030009EBA03D0F2A4FCD703D00050AE5C02E00D
:10104000000E01D0010E41E9E7CFD9FF1200DCD834
:1010500083E944E880EB04F081EB05F0010E066EB5
:101060008A8400EBE9FF01EBEAFFEF04036E03342F
:1010700020E2ACA2FED7042A000E052204EBE9FF11
:1010800005EBEAFFEF50AD6E04EBE9FF05EBEAFF7D
:10109000EFCFE6FFC6DF41E9000902E1066A09D0A9
:1010A000033405E20350000802E22A0EB2D8030618
:1010B000DED78A94065045E9E7CFD9FF1200A4D8BD
:1010C00086E945E8066A83EB09F084EB0AF0F294BE
:1010D0000150AE0802E2AE0E016E0150000181D84F
:1010E000C6C0C5F0C66BC5C0D7FF01507AD8C55180
:1010F000D66E5ED8C6C0C5F0C66BC551076E58D84F
:10110000C551086E03EBE9FF04EBEAFFEF6A066ADC
:101110000250065C19E29EBA03D0F2A4FCD714D0A8
:10112000ABB412D0ABB210D0092A000E0A2209EBE0
:10113000E9FF0AEBEAFFAECFEFFF8A8207EBD7FFAA
:1011400008EBD6FF062AE4D703EBE9FF04EBEAFF3E
:1011500006EBEFFF8A9246E9E7CFD9FF12008A84B7
:10116000AB9EAC9A1BD81AD85FD8AB8EAC8A8A9447
:1011700082AE000C010C8A84AB9EAC9A8B9C8A8652
:101180008A8A960E46D88B8C8A968A9A960E41D871
:10119000AB8EAC8A8A9482AE000C010C45D88B8C45
:1011A0008A968A9A3BD88B9C8A868A8A0EEF09F0A7
:1011B000040EE66EE66A770EE66E010EE66E0050ED
:1011C000E66EE66AEFEC0BF0B3EC0BF0E552E5CF20
:1011D000C6F0E7CFC5F00001FF0ED880C557C6574F
:1011E0001200C56FC66B770EC603F3CFC6F0C551AC
:1011F000C627770EC503F3CFC5F0F450C627FF0E00
:10120000D880C557C6571200D9CFE6FFE1CFD9FF26
:101210001200E66E60EC0FF041E91200780EE66E07
:1012200045EC0FF041E912008B9C8A868A8AF6DF32
:0A1230008B8C8A968A9A0EEF09F063
:06123A000001CA51CB11B6
:1012400004E1100ECA6F270ECB6FCA07000ECB5BEE
:101250006DA205D0CA51CB1116E18A7012000001AF
:10126000C151060A0FE0030A0BE0060A09E0010A71
:101270000AE0030A05E0010A01E012008A90120068
:101280008A8012008A801200D9CFE6FFE1CFD9FF11
:1012900081E945E8D2DF060E0001C15D64E36D50CF
:1012A000020B61E1ACD8A5EC0AF042E9F350016E03
:1012B000F450026E5A0E0124036E000E0220046EDA
:1012C000000101502908C56F000E0254C66FC5C049
:1012D000E6FF03EBE6FF04EBE6FFA9EC04F043E9CD
:1012E000000941E000018351056E05500126000E02
:1012F0000222290E015C000E025833E25A0E01242C
:10130000E96E000E0220EA6EEF6A000100A306D02B
:1013100003EBE6FF04EBE6FF35D842E90D0EE66E7F
:101320006ED85AEC0AF043E9F350036EF450046EA1
:101330000350041018E000010051020B09E00051B5
:10134000080B06E06C0EE66E1D0EE66E2ED842E926
:1013500003EBE9FF04EBEAFFEF6A51D868EC03F016
:1013600042E900015A6B46E9E7CFD9FF12000001BC
:101370005A6B12005FEC0CF06FBE02D07BEC0CF0ED
:1013800005EF05F033D80001845103E021D8FBE2DA
:1013900008D000EBE6FF01EBE6FFDAEC04F042E9EF
:1013A000E9DF43E9E7CFD9FF120020D800018451DB
:1013B00003E00ED8FBE208D000EBE6FF01EBE6FF0E
:1013C000EFEC04F042E9D6DF43E9E7CFD9FF1200A2
:1013D000D1DF032A000E042203EBC5F004EBC6F0B4
:1013E0000001C551E808030EC6551200D9CFE6FF2B
:1013F000E1CFD9FF83E942E8036A046A12005A0E7A
:08140000E66E000EE66E12001C
:08140800FC0EE3CFF6FFFD0E20
:10141000E3CFF7FFFE0EE3CFE9FFFF0EE3CFEAFFD6
:10142000FA0EE35003E1FB0EE35009E0FA0EE30687
:1014300002E2FB0EE3060900F550EE5CF1E0F36E0C
:101440001200FC0EE3CFF6FFFD0EE3CFF7FFFE0E1A
:10145000E3CFE9FFFF0EE3CFEAFFE9CFF3FFEACFE7
:10146000F4FFFA0EE35003E1FB0EE35009E0FA0E3D
:10147000E30602E2FB0EE3060900F5CFEEFFF1D72B
:101480001200FC0EE3CFF6FFFD0EE3CFF7FFFE0EDA
:10149000E3CFE9FFFF0EE3CFEAFFE9CFF3FFEACFA7
:1014A000F4FFEE66FED7ED520900F5CFEFFFEE66D2
:1014B000FBD71200FE0EE3CFE9FFFF0EE3CFEAFFFA
:1014C000FD0EE350EF5C05E0EE66FAD7F36AF46ACE
:1014D00004D0E9CFF3FFEACFF4FF1200D9CFE6FF43
:1014E000DACFE6FFFA0EE3CFD9FFFB0EE3CFDAFF48
:1014F000FC0EE3CFE9FFFD0EE3CFEAFFE9CFF3FFF8
:10150000EACFF4FFDECFEFFFEE66FCD7FF0EE3CFAE
:10151000DAFFE552FF0EE3CFD9FFE5521200FC0ED1
:10152000E3CFF6FFFD0EE3CFF7FFFE0EE3CFE9FFBB
:10153000FF0EE3CFEAFFE9CFF3FFEACFF4FF0900A4
:10154000F5CFEFFFEE66FBD71200FE0EE3CFE9FF0B
:10155000FF0EE3CFEAFFF36AF46AEE5203E0F34AC8
:10156000F42AFBD71200FF0EE3CFF7FFE552FF0E80
:10157000E3CFF6FFE552E56AE66AE66AE66A090045
:10158000F55209E0FD0EE32A05E1FE0EE32A02E131
:10159000FF0EE32AF4D7FD0EE3CFBDF0FE0EE3CF3E
:1015A000BEF0FF0EE3CFBFF01200FE0EE3CFE9FF67
:1015B000FF0EE3CFEAFFE9CFF3FFEACFF4FF610EBE
:1015C000EF5C05E67B0EEF5C02E7DF0EEF16EE52F6
:0415D000F6E112002E
:0C15D400FE0EE3CFE9FFFF0EE3CFEAFFBD
:1015E000EFCFF3FF030EEF26F36EE926000EEA229B
:1015F000040EEDCFEBFFF32EFCD7680EEC6E6A0EF7
:10160000EC6EF10EEC6EFD0EEB501200FE0EE3CF11
:10161000E9FFFF0EE3CFEAFFEFCFF3FFF3CFF4FFD5
:10162000F42AF4CFEEFFE86AEE24F32EFDD7EF6E36
:10163000F4501200FE0EE3CFE9FFFF0EE3CFEAFF06
:10164000EFCFF3FF030EF35E0AE009E6F3CFF4FFFA
:10165000F3CFEEFF030EEBCFEEFFF32EFCD7F450EB
:101660001200FE0EE3CFE9FFFF0EE3CFEAFFEFCF5C
:10167000F3FFF306F3CFF4FFF3CFEEFFE86AEE24B7
:10168000F32EFDD7EF18D8B4F4501200D9CFE6FFEF
:10169000DACFE6FFFC0EE3CFE9FFFD0EE3CFEAFF72
:1016A000F90EE3CFF4FFEFCFF3FFEF50E926000E82
:1016B000EA22030EF4B0E82AD96EE82AEDCFEBFF58
:1016C000F32EFCD7EFCFF3FFD950EF26FA0EE3CF7E
:1016D000D9FFFB0EE3CFDAFFE86AF4A0F350DE1087
:1016E000EC6EDECFECFFDECFECFFF4B0F3CFECFF1F
:1016F000E552E7CFDAFFE552E7CFD9FFF4B002D0E9
:10170000FD0E01D0FC0EEB501200D9CFE6FFFD0E0E
:10171000E3CFE9FFFE0EE3CFEAFFEFCFF3FF010EC9
:10172000EB503F0B030ED8B4E82AD96EF35E0AE003
:1017300009E6F3CFF4FFF3CFEEFFD950EBCFEEFF86
:0E174000F32EFCD7E552E7CFD9FFF45012008C
:02174E0043E86E
:10175000D9CFE6FFDACFE6FFE1CFD9FFE2CFDAFF5C
:1017600089E9066A1200F3DF068001D0F0DF01AEDE
:10177000C0EF0BF0006C011EE86A012206B0067E85
:1017800003AEC8EF0BF0026C031EE86A0322067E6C
:1017900034EC0CF003BEEAEF0BF006AE08D0026C9E
:1017A000031EE86A0322046C051EE86A052206B0DF
:1017B00006D084EB00F085EB01F006A004D082EBAC
:1017C00000F083EB01F0E552E5CFDAFFE7CFD9FF78
:1017D00045E9000C06BECFEF0BF0E9DFFF0C44E853
:1017E000D9CFE6FFDACFE6FFE1CFD9FFE2CFDAFFCC
:1017F0008AE980EB04F081EB05F082EB06F0025001
:101800000402F450016EF350006E0350076E05029F
:10181000F450036EF350026E07500402F350012699
:10182000F4500222E86A032206500502F350012612
:10183000F4500222E86A0322E552E5CFDAFFE7CF4F
:10184000D9FF46E9000C43E8D9CFE6FFDACFE6FF3F
:10185000E1CFD9FFE2CFDAFF89E9066A1200F3DFB0
:10186000068003D0F0DF01D00682056A046A100EFC
:10187000E76ED89002360336043605360050045C15
:101880000150055805E30050045E0150055A022A34
:10189000E72EF0D706B2120006B006D084EB00F0B7
:1018A00085EB01F006A004D082EB00F083EB01F0A1
:0E18B000E552E5CFDAFFE7CFD9FF45E9120098
:0218BE006DA615
:1018C0000CD80001C10508E16DBA06D0686A696AE2
:1018D00069806988020EC16F12006D6A696A6D863F
:1018E0000001010EC16F12006D6A696A0001C16BCF
:1018F000120074EF0CF00001C15101E112006850B8
:10190000040B04E06950040B01E038D86DB21200FA
:101910006850010B04E06950010B01E050D8685099
:10192000100B04E06950100B01E024D86850400B04
:1019300004E06950400B01E037D86850200B04E008
:101940006950200B01E032D86850020B04E0695066
:10195000020B01E032D8030E0001C15D01E212006A
:101960006850080B06E06950080B03E0D4EC06F061
:1019700068961200698468986D8212006D9269946D
:10198000689412000001C2A10ED0F8DF6D8400013E
:10199000080EC86F070EC96FC807000EC95BC85193
:1019A000C911FAE16D941200689C120070A003D076
:1019B000DFEC07F07090689A1200689212006A6A71
:1019C000686A9F0E6B6E7B0E696E6E6A0F0EE66E16
:1019D000710EE66E0F0EE66E12D843E9160E706EAB
:1019E00068A602D06896FCD76D98DFEC07F000017E
:1019F000C2910001C36B0001030EC16F1200D9CF69
:101A0000E6FFE1CFD9FF84E901EBE9FF02EBEAFF52
:101A1000005003E0EE6A0006FBD741E9E7CFD9FFAB
:021A20001200B2
:0E1A2200FE0EE3CFE9FFFF0EE3CFEAFFF36A0B
:101A3000EE5006E018D8FCE009D806E1F32AF8D702
:101A4000F3B002D0F3501200E86A1200F452C60F4D
:101A50000A0F06E2F450B90F060F02E2D894120002
:101A6000F450D8841200F46E200806E0F4500908FF
:101A700003E0F450D8941200D8841200D9CFE6FFC6
:101A8000DACFE6FFFC0EE3CFE9FFFD0EE3CFEAFF7E
:101A9000FC0EE3CFD9FFFD0EE3CFDAFFF36ADE5091
:101AA00007E0E1DFFCE0D2DF1FE1F32AEE6EF7D7BB
:101AB000EF6AF3B019D0F342FC0EE3CFE9FFFD0E5D
:101AC000E3CFEAFFFA0EE3CFD9FFFB0EE3CFDAFF55
:101AD000F3CFDEFFEF5206E00FD8E83ADF6E0CD806
:101AE000DE12F8D7F35001D0E86AE552E7CFDAFF0B
:101AF000E552E7CFD9FF1200EE50C00FD8A0070F74
:101B0000090F1200D9CFE6FFDACFE6FFFC0EE3CFD4
:101B1000E9FFFD0EE3CFEAFFFB0EE3CFF3FFF90E83
:101B2000E3CFD9FFFA0EE3CFDAFFF3520FE0EF5025
:101B3000F00BE83A12D8DE6EEE500F0B0ED8DE6EC8
:101B4000200EDE6EF32EF3D7DD52DF6AE552E7CFCB
:101B5000DAFFE552E7CFD9FF1200360FD8B2070FF0
:041B6000FA0F120066
:0C1B64004F4244444941472E4E45542056
:101B700076312E323520627920416C6578205369A8
:101B8000646F72656E6B6F2C20504943313846325A
:101B9000343530003F004F4B00454C4D333233203D
:101BA00076322E3020636F6D70617469626C6500EF
:101BB00044415441204552524F52003C444154410B
:101BC000204552524F52004E4F204441544100454F
:101BD00052524F52004642204552524F52004255F7
:101BE0005320425553590050726F6772616D204502
:101BF00072726F7200D81DD31DCF1DCA1DC51DC0C6
:101C00001DBB1DB61DB11DAD1DA81DA31D9E1D999B
:0F1C10001D941D8F1D8A1D851D801D7C1D771D38
:011C1F0012B2
:101C200001000202000008D8040A000000010203BB
:101C30000109024300020100803209040000010290
:101C400002010005240010010424020205240600FC
:101C500001052401000107058203080002090401AF
:101C600000020A0000000705030240000007058388
:101C7000024000000403090418034F0062006400DE
:101C800044006900610067002E004E00650074008A
:101C90001A034F004200440032002000410064005B
:101CA0006100700074006500720016033100370097
:101CB000340031003500310032003400350030008E
:0E1CC000311C311C741C781C901CAA1C5E0880
:021CCE002A0EDC
:101CD000F66E000EF76E000EF86E00010900F5506A
:101CE000B06F0900F550B16F03E1B06701D03DD08E
:101CF0000900F550AB6F0900F550AC6F0900F550C5
:101D0000AD6F09000900F550E96E0900F550EA6E63
:101D1000090009000900F550AE6F0900F550AF6FDA
:101D200009000900F6CFB2F0F7CFB3F0F8CFB4F066
:101D3000ABC0F6FFACC0F7FFADC0F8FF0001AE537B
:101D400002E1AF5307E00900F550EE6EAE07F8E28E
:101D5000AF07F9D7B2C0F6FFB3C0F7FFB4C0F8FFC2
:0C1D60000001B007000EB15BBFD71200FD
:041D6C000A000A005F
:101D70000D004154003E00415440310041545A008E
:101D8000415453570041545354004154535200415D
:101D90005453490041545348004154504400415465
:101DA0004D410041544C310041544C3000415449A4
:101DB00000415448310041544830004154464900E4
:101DC000415446440041544531004154453000419E
:0D1DD000544400415442440041544152002B
:021DDE00D9CF5B
:101DE000E6FFE1CFD9FF84E9AC6AAB6A02A005D077
:101DF000AC8802A404D0AC8E02D002B8AC8402A29B
:101E000002D0AC8CAB8C02A602D0AB8801D0AB8ADE
:101E100002AC02D09D8A01D09D9A02AE02D09D886C
:101E200001D09D9800EBAFFF000101EBC5F0C66B40
:101E3000C5C0B0FFAC8AAB8E41E9E7CFD9FF120035
:101E40000F0EC112C00E8A169316800E946EF29E6B
:101E5000F29C850ED56EF28AB50ECD6E9D80120075
:101E6000140E6F6E0001C16B0001C26B0001C36BE9
:101E7000E7DFB7EC09F0C2EF03F0F2DFBAEC09F0EC
:0A1E800044EC09F054EC01F0F9D72E
:061E8A00FF0EE350000111
:101E9000CD6FEE0E02D0F20E0000E76EE72E4EEF91
:101EA0000FF00C0E0001CC6FE76AE72E55EF0FF034
:101EB000CC2F54EF0FF00001CD2F4BEF0FF012009D
:101EC000FF0EE3500001CD6F480E01D04C0EE76EBF
:101ED000E72EFED7E76AE72EFED7CD2FF7D7120001
:101EE00011EE00F021EE00F0F86A67EC0EF090ECD5
:0A1EF0000FF03DEC0FF0FBD71200DD
:061EFA000181020100005D
:101F0000013E425553494E49543A20002E004F4B52
:011F100000D0
:0E1F120000EE00F00F0EEE6AEA62FDD712003C
:021F20001200AD
:021F22000000BD
:020000040030CA
:0100000034CB
:010001000EF0
:010002003FBE
:010003001EDE
:0100040000FB
:01000500807A
:01000600C138
:0100070000F8
:0100080000F7
:0100090000F6
:01000A0003F2
:01000B006094
:01000C0003F0
:01000D0040B2
:00000001FF
